:020000020000FC
:1000000004C01895FFC0FBC0FCC0789450E25BBFF1
:10001000442445BE41BC4CBA6624639402E009BF47
:1000200005E003BF00E808B900E308BB08E007BB30
:1000300000E2502E40EC76B204E00EBBE09A0DB325
:100040000C3601F1033CE9F00E39E9F0242CE1997A
:10005000FECFF894A5E0AEBB2DBAE29AE19A78946F
:10006000E199FECF27C1466F786F5458204153382D
:1000700030342028632920444A32544B2056322EF3
:10008000326318C116C0E199FECFF894A4E0AEBB6C
:10009000ACE6ADBBE29AE19A7894E199FECF00C05C
:1000A00066275BBF689495D094D093D00FEF44BE81
:1000B0001DC044BE05E00EBBE09A0DB3202E239474
:1000C000E199FECFF894A5E0AEBB2DBAE29AE19A91
:1000D0007894E199FECF322C15E09AE47AD09A9583
:1000E000E9F71A95D1F73A94B9F7DACF3EF4D0E0B0
:1000F000C4EF04C065A858A222960300FD2FEC2F80
:10010000C8953327079440F0079420F062D061D05F
:1001100060D022C06BD020C0079410F05ED01CC00D
:1001200058D057D056D055D054D06F3F09F40895C9
:10013000CEF0EC2FFD2F83958E3101F788272224F6
:10014000E199FECFF894A5E0AEBB2DBAE29AE19A10
:100150007894E199FECFD2CF3395343098F2E60D02
:10016000F41DCECFE894D1E0CEE74EBAE09A0DB3BD
:100170000F3F21F2C00FD41DC00FD41DBFCF3900D7
:1001800056036603D6000D006503DA0055033500FB
:10019000A903E60059033A003600EA0069039A030E
:1001A000D900D5000E00E5009503E9009603A603EB
:1001B0005A03AA0EA90EA50E950E550E550D560DF5
:1001C0005A0D6A0DAA0DA535960D563999395A3A28
:1001D000560E42BF55BE88950895C39A22E042BF8D
:1001E00055BE88952A95D9F7C398F3CFC39A24E0D2
:1001F00042BF55BE88952A95D9F7C398EACF42BF2A
:100200001895189586B2872476B284FE189574FCEA
:100210001895A2E0A9BF7894A4E0AEBBE09AADB374
:10022000A33CD9F44BBED5DFB49944C0D2DFB49916
:1002300041C0CFDFB4993EC0D0DFCFDFB49BFECF4B
:10024000E199FECFF894A4E0AEBBAEE9ADBBE29A73
:10025000E19A7894E199FECFD8CE4BBE4ABEB9DF81
:10026000B8DFBBDFB6DFB5DFB4DFB3DFB2DFB1DFEE
:10027000B4DFB3DFB49914CFACDFABDFAADFA9DF03
:10028000A8DFA7DFA6DFA9DFA8DFA7DFB49926C014
:10029000A0DF9FDF9EDF9DDF9CDF9BDF9ADFB499AD
:1002A00041C081D096DF95DFB49BFECF92DF95DF12
:1002B00094DF8FDFE199FECFF894A4E0AEBBA3EC0E
:1002C000ADBBE29AE19A7894E199FECF4ABE48BE6E
:1002D0005BBF49BE00E305BF889597CE6FEF79DF1E
:1002E00078DF77DF76DF742DD1E0CEE7C70FD41D3E
:1002F000C70FD41D03DF02DFB49B04C073957A32AD
:1003000099F7CECEE199FECFF8944EBA7DBBE29A32
:10031000E19A7894E199FECF33D05BDFB49BFECFB6
:1003200058DFBECE6FEF55DF54DF53DF52DF0027BB
:10033000D1E0C2EBC00FD41DC00FD41DDFDEDEDE66
:10034000B49B04C003950A3099F7AACE23D0B49B7E
:10035000FECF3FDFF3E0E6E7E00FF41DC8954ABEAD
:100360005BBFEDE1FFEF35DFFA95E9F7EA95D1F7ED
:100370000A94B9F795CE010204070A0D131F49919B
:1003800028DF2BDF33DF29DF24DF23DF22DF21DF3C
:1003900020DF86CE1EDF21DF29DF1FDF1ADF19DF16
:1003A00018DF17DF089519DF18DF17DF1FDF15DFEC
:0403B0001DDF0895B0
:00000001FF
